:100000000C94F0030C9489000C94970018951895A3
:100010001895189518951895189518951895189578
:100020001895189518951895189518950C94A5007D
:100030000C9475001895189518951895189518959D
:100040001895189518951895189518951895189548
:10005000189518951895189508D00CE211E097D3CB
:1000600014D02AD030D095D008950FEF0ABB0BBB27
:100070000EE407BB0EE008BB03EE04BB0FEF05BBAD
:1000800000EF01BB0CEF02BB089500E00FB90CE4D8
:100090000DB96F9A0EB10FB10AB700640ABF05B768
:1000A000026005BF0BB700640BBF0AB700680ABF48
:1000B00005B70C6005BF089505E003BF01E008BF68
:1000C0000AEF02BF089501EA0FBD02E605BD00E098
:1000D0000DBD0CBD04BD0BBD0FEF0ABD00E009BD99
:1000E0000FEF08BD03BD789408952A931A930A93DD
:1000F0002FB71FB701E00093A6000FB10093A50032
:100100000091A7000FB91FBF2FBF09911991299125
:1001100018952A931A930A932FB71FB701E00093FB
:10012000A0001FBF2FBF09911991299118952A93FB
:100130001A930A932FB71FB701E00093A0001FBFC7
:100140002FBF0991199129911895FA93EA934A932F
:100150003A932A931A930A934FB71FB7E3EAF0E052
:10016000208131812F5F3F4F208331830AEF02BF0F
:100170001FBF4FBF09911991299139914991E99177
:10018000F9911895E199FECF0EBB1FBBE09A0DB314
:1001900008950E940204239781E000E00093A100EB
:1001A000E3EAF0E00083018301C0EDD20091A600F4
:1001B000002309F049C003B30C700093A80000911C
:1001C000A800043029F4E7EAF0E000810E7F008304
:1001D0000091A800002321F00091A800002329F439
:1001E000E7EAF0E00081016000830091A7000FB909
:1001F0008130D9F2A13011F5A0E0A093A2000B2F1D
:100200000F700B3018F40B2F0F7033D10B2F0073BE
:1002100019F00B2F00733FD1B09B05C0E7EAF0E067
:1002200000810D7F0083B09905C0E7EAF0E000810E
:10023000026000830091A7000FB9B8CF913009F098
:10024000B5CF8E0172D0B2CFB091A5000B2F007C3C
:10025000005889F00054C1F0005419F0005409F01E
:10026000A5CF08B30E6008BB00E00093A60081E0B4
:10027000A0E090E09BCF08B30E6008BB00E00093C5
:10028000A60080E0A1E0F5CF0B2F0ED008830B2F46
:1002900020D009830B2F33D00A8300E00093A600FF
:1002A00080E0A0E091E082CF2397007339F0005105
:1002B00039F0005139F0005139F008C008E005C0AC
:1002C00005E003C002E001C000E008830881239636
:1002D000089523970C7039F0045041F0045041F018
:1002E000045041F009C0C29A0AE005C005E003C00D
:1002F00002E001C000E00983098123960895239755
:10030000037039F00A9541F00A9541F00A9541F0E1
:1003100009C0C19A0AE005C005E003C002E001C0BF
:1003200000E00A830A8123960895192E282EF801E9
:100330005FEF3FEF1FEF6FEF8081805039F0825009
:1003400059F0835031F0835051F00BC001E057EF6A
:1003500008C041E037EF05C021E017EF02C071E0AF
:1003600067EF8091A200843618F18181805029F0D6
:10037000825049F0835021F008C001E05B7F05C046
:1003800041E03B7F02C021E01B7F8281805029F049
:10039000825049F0835021F008C001E05D7F05C024
:1003A00041E03D7F02C021E01D7FE5E6E093A20031
:1003B000E0E0E093A0000090A0000020E1F3E2EA7A
:1003C000F0E0808183958083013019F408B3052320
:1003D00008BB4130B9F40091A100013021F400E0E4
:1003E0000093A1000FC008B3032308BB00E004C0C2
:1003F00041E04093A10003950A30D0F3309508B353
:10040000032B08BB40E0E3EAF0E040834183213066
:10041000A1F409B7016009BF8081918183309040C8
:10042000DCF308B3012308BB00E001C003950A30E8
:10043000E8F3109508B3012B08BB7130A1F409B79C
:10044000016009BF8081918189309040DCF308B35D
:10045000062308BB00E001C003950A30E8F360956D
:1004600008B3062B08BB09B70E7F09BF822D912D5B
:100470000895023058F00A3019F400E003BD0895E1
:100480001FEF29E1029F101913BD0895013011F4E7
:100490000FEF03BD08950E940204902F8FEF00918B
:1004A000B100002309F488D102E00EBD0FEF67D13F
:1004B0000FEF67D103B30C700093A800903109F0DF
:1004C0009AC00091A800043021F00091A8000C30DF
:1004D000B1F50091A800043041F4E7EAF0E00081B2
:1004E0000E7F00830091A7000FB900E0E3EAF0E07F
:1004F000008301838091A90009B7016009BF11C081
:100500008A95082F3CD10FEF3CD10091AA0010E052
:10051000E3EAF0E02081318102171307B4F710837A
:100520001183882369F709B70E7F09BF04C003B39D
:100530000C700093A8000091A8000830C1F700914A
:10054000A800083071F480E000E019D10FEF19D154
:1005500004C003B30C700093A8000091A80000230E
:10056000C1F70091A800002309F041C000E0E3EAD0
:10057000F0E00083018309B7016009BF0091B10079
:10058000002331F50EC0082FFAD00FEFFAD0839573
:10059000E3EAF0E0A081B1811697D4F300E0008394
:1005A0000183853B80F301E00093B10015C0082F63
:1005B000E6D00FEFE6D083950091AC0010E0E3EABF
:1005C000F0E02081318102171307B4F71083118303
:1005D0000091AB00081758F7E7EAF0E000810160EE
:1005E00000830091A7000FB909B70E7F09BF0FEF75
:1005F000C6D00FEFC6D0903209F0A0C089E10091BB
:10060000A800002321F00091A8000023B1F500917B
:10061000A800002341F4E7EAF0E0008101600083D4
:100620000091A7000FB900E0E3EAF0E00083018346
:100630008091AD0009B7016009BF11C08A95082FEC
:10064000A0D00FEF9CD00091AE0010E0E3EAF0E004
:100650002081318102171307B4F710831183882397
:1006600069F709B70E7F09BF04C003B30C7000938C
:10067000A8000091A8000830C1F70091A800083038
:10068000B1F4E7EAF0E00081016000830091A70087
:100690000FB980E000E075D00FEF71D004C003B354
:1006A0000C700093A8000091A8000C30C1F70091D5
:1006B000A8000C3099F5E7EAF0E0008101600083C2
:1006C0000091A7000FB9893119F400ED17E05FD050
:1006D00000E0E3EAF0E00083018309B7016009BFAD
:1006E00011C08395082F4DD00FEF49D00091B00075
:1006F00010E0E3EAF0E02081318102171307B4F73C
:10070000108311830091AF00801758F309B70E7F53
:1007100009BF04C003B30C700093A8000091A800A7
:100720000430C1F7E7EAF0E000810E7F008300911A
:10073000A7000FB90FEF25D00FEF21D000E010E098
:10074000E3EAF0E00083018309B7016009BFA3EA8F
:10075000B0E0ED91FC913597D4F3E3EAF0E010833B
:10076000118309B70E7F09BF0EB50D7F0EBD00EFD7
:1007700001BB02B3006302BBE4E00C9407040ABDB2
:10078000089508BD089500E00093A2000895392F50
:10079000482FE0E0F0E007C000000196883522E035
:1007A0009207D4F33196E017F1071CF480E090E053
:1007B000F5CF842F932F08959A938A93F89480E02D
:1007C00009C0082F10E0DEDC90E0FC01E755FF4F88
:1007D000008383958830A8F378948991999108953E
:1007E0000FE90DBF00E00EBFC0E8D0E00E94120488
:1007F000002311F00E9422040E942C000E943C045D
:100800000C943C04BA93AA939A938A930895BB815B
:10081000AA8199818881F0E00FB6F894CE0FDF1F8E
:100820000FBE089501E0089520E002D0E9F7089591
:100830002D9301501040202F212B08952591F8DF92
:10084000E9F708958EE798E0FC0105911491FC0109
:100850003296A591B491FC01349625913491422FA2
:10086000432B19F0F901EADF01C0DEDF069618E03C
:100870008438910748F3089500008895FECF120050
:04088000A0000000D4
:00000001FF
